:020000020000FC
:0200000070C1CD
:0200040018954D
:02000800189549
:02000C00189545
:02001000189541
:0200140018953D
:02001800189539
:02001C00189535
:02002000189531
:0200240018952D
:02002800189529
:02002C00189525
:02003000189521
:0200340018951D
:02003800189519
:02003C00189515
:02004000189511
:0200440018950D
:02004800189509
:02004C00189505
:02005000189501
:020054001895FD
:020058001895F9
:02005C001895F5
:020060001895F1
:100064001895FF1829E0001F2A9509F40895FF1C2C
:10007400F11A18F4F10E8894F6CF0894F4CF5F9A2D
:1000840000FF5D9800FD5D9A01FF5C9801FD5C9A9C
:1000940002FF5B9802FD5B9A03FF5A9803FD5A9A8C
:1000A4005F9808955E9A0F930295E9DF0F91E7DF59
:1000B400BB27AAEF58D008955E980F930295DFDF0F
:1000C4000F91DDDF02E052D008950591003011F068
:1000D400E9DFFBCF08950A3020F017E3010FE2DFD8
:1000E400089510E3010FDEDF08951F930F93029527
:1000F4000F70F1DF0F910F70EEDF1F910895EE2462
:100104001AE0AFDFE394FF920030D1F710E30F91D0
:10011400010FC8DFEA94D1F708950068CDDF089590
:100124000064CADF0895559A549A539A529A569A7B
:10013400579A5E985F9804E619D013E003E09FDFB6
:1001440005E014D01A95D1F702E099DF01E00ED052
:1001540008E2B2DF08E0B0DF01E0AEDF06E0ACDFCA
:100164000CE0AADF08951197F1F708950F93B7E013
:10017400A0EDF9DFB7E0A0EDF6DF0A95C1F70F9126
:1001840008952898209AB7E0A8E5EDDF2098B1E01B
:10019400A8E1E9DF6894189BE894B3E0A0ECE3DFFE
:1001A400089518F4B0E0A4E002C0B1E0A0EE209AF3
:1001B400DADF2098B0E0A0EFD6DF08951F9310E0B7
:1001C4000795EFDF13951830D9F71F910895B0E024
:1001D400A4E0209AC8DF2098B0E0A4E1C4DFE8944A
:1001E40018996894B0E0A8ECBEDF08940EF08894E7
:1001F40008951F9310E0EBDF079513951830D9F796
:100204001F910895C8E0D1E0BCDFE6F3BADFD6F36E
:10021400B8DFC6F30CECD2DF0EEBD0DFEADF0993D4
:10022400502FE7DF0993602F0895ABDF5EF30CECEA
:10023400C5DF04E4C3DF0CEB99DF18950F931F931C
:10024400C8E0D1E0A991B991A695A69503E02A2F1B
:10025400202309E1209F9001A695A6950FE0B023E5
:10026400B795B795B795B795B795AB2B1F910F91E8
:1002740008950F931F932F930F9318E0209110016B
:10028400022707950091100110F428E10227079531
:10029400009310010F9106950F931A9579F70F911A
:1002A4002F911F910F9108950F9300E00093100177
:1002B4000F91089500911001089569427574746F47
:1002C4006E2052656164657200006176722D6D6303
:1002D400752E6478702E706C00002E0000000FEFF5
:1002E4000DBF21DF01E019DFEEEBF2E0EEDE01E409
:1002F40014DF47DFF6F30CEC61DF0EE45FDF002769
:100304005DDF5CDF0FE35ADF01E407DF3ADFE6F38A
:100314008CDF78DF93DF0C94A4016BDF0030A1F352
:10032400A8DFC0E0D1E0099317E063DFA2DF0993FF
:100334001A95D9F7BFDF003039F700E4EEDEC0E0EC
:10034400D1E012E00F930A2F0F9330EF032320D054
:100354000695069506950695BEDE0F9119D02FE0F9
:100364000223B9DE022F0F9330EF032311D0069539
:10037400069506950695AFDE0F910AD02FE002236D
:10038400AADE0000000000000C948601D9F6BCCF60
:1003940055270A5010F0505FFCCF065F050F0895F3
:00000001FF
